:0200000480007A
:100000006F000005732F2034930F80006308FF03F7
:10001000930F90006304FF03930FB0006300FF038E
:10002000130F000063040F0067000F00732F2034CC
:1000300063540F006F00400093E19153171F0000BD
:1000400023223FFC171F000023200FFC6FF01FFF2F
:100050009300000013010000930100001302000050
:100060009302000013030000930300001304000038
:100070009304000013050000930500001306000020
:100080009306000013070000930700001308000008
:10009000930800001309000093090000130A0000F0
:1000A000930A0000130B0000930B0000130C0000D8
:1000B000930C0000130D0000930D0000130E0000C0
:1000C000930E0000130F0000930F0000732540F102
:1000D0006310050097020000938202017390523072
:1000E000735044749702000093820201739052305F
:1000F00073500018970200009382420273905230AE
:100100009B021000939252039382F2FF7390023B82
:100110009302F0017390023A73504030970200004E
:1001200093824201739052307350203073503030BC
:100130009301000097020000938202ED7390523009
:10014000130510001315F501635C05000F00F00F97
:10015000930110009308D005130500007300000000
:1001600093020000638A020073905210B7B200003D
:100170009B829210739022307350003097020000DF
:100180009382420173901234732540F17300203042
:10019000930120003705008093050080972600001A
:1001A000938646E623A0A6002FA7B6A0B70300803B
:1001B000631C77069301300083A706009303008039
:1001C00063947706930140009305100023A0060076
:1001D0002FA7B6A093030000631877049301500083
:1001E00083A70600930310006390770493016000D7
:1001F000130510009B0510009395F501972600004C
:10020000938646E023A0A6002FA7B6A09303100074
:10021000631C77009301700083A70600930310000E
:1002200063947700631030020F00F00F63800100C9
:100230009391110093E111009308D00513850100FB
:10024000730000000F00F00F930110009308D00519
:100250001305000073000000731000C000000000D0
:10026000000000000000000000000000000000008E
:0C02700000000000000000000000000082
:1010000000000000000000000000000000000000E0
:1010100000000000000000000000000000000000D0
:1010200000000000000000000000000000000000C0
:1010300000000000000000000000000000000000B0
:081040000000000000000000A8
:040000058000000077
:00000001FF
